:0C000000830100308A00042883015F2A7D
:10048400A000831289008316081483120808080048
:100494000800A100831688184D2A210883128900B8
:1004A400200888008B138316081555308900AA305C
:1004B4008900881408118312080083168601FF300E
:1004C40085008E018F01013083124222960097012C
:1004D4000230422298009901940195019E019F01E6
:1004E40005088C008D010A30900091010D08A300CD
:1004F4000C08A2000230A205A3012208023A230438
:10050400031D852A862A8E2A9801990100309600B7
:100514000130970080308600ED2A0D088312A30075
:100524000C08A2000130A205A30122032304031D29
:100534009C2A9D2AA12A8E0A03198F0AD12A0F0800
:100544000E04031DA62AA72AA82AD12A1908803A2C
:100554008312A2000F08803A2202031DB32A0E0858
:1005640018020318B62AB72ABC2A0E0898000F08E6
:100574009900CF2A0F08803A8312A2001708803A04
:100584002202031DC72A16080E020318CA2ACB2A00
:10059400CF2A0E0896000F0897008E018F011E08BF
:1005A4000A3A1F04031DD72AD82AD82A8312050819
:1005B4008C008D018C18DF2AE02AED2AFD30960785
:1005C400031C97031608A000013083124B2218085D
:1005D400A00002304B220D088312A3000C08A200D5
:1005E4000230A205A3012208023A23040319FB2ABC
:1005F400FC2A8F2A02308312A4000030A5001908B7
:10060400A3001808A2001608A202031CA3031708DB
:10061400A3020330A2070318A30A0030A307B423DC
:1006240026089A0027089B00F6301A079000FF302E
:10063400031800301B07910003309C009D01B22B6E
:10064400831205088C008D010C1C292B2A2B2E2BC0
:100654008E0A03198F0A8A2B0F080E040319332BF1
:10066400342B8A2B16080E0292001708031C170A53
:100674000F029300931F3F2B402B432B92019301B6
:10068400882B1B08803A8312A2001308803A2202A6
:10069400031D4E2B12081A020318512B522B6C2BDC
:1006A4001A089202031C93031B0893021308803A4E
:1006B400A2001D08803A2202031D622B1C081202AC
:1006C4000318652B662B682B920193019401940AFD
:1006D4009501882B12081A0292001308031C130AAE
:1006E4001B0293001308803A8312A2001D08803A6B
:1006F4002202031D7F2B1C0812020318822B832B5A
:10070400852B920193010230940095018E018F0193
:100714001F08803A8312A2001308803A2202031DA4
:10072400952B12081E020318982B992B9C2B140846
:1007340086009E2B831286019E0A03199F0A1108C4
:10074400803A8312A2001F08803A2202031DAC2BB8
:100754001E0810020318AF2BB02BB22B9E019F0171
:10076400222B0428A801A31FBE2BA209A20A031945
:10077400A303A3092817A81725088039A806A51FCD
:10078400CA2BA409A40A0319A503A509CA2BA80105
:10079400A601A70124082504031900341F30A80466
:1007A4000310A80AA40DA50D031CD32BA50CA40C9F
:1007B40025082302031DE02B24082202031CE82B36
:1007C4002408A2022508031C250AA302A60DA70DCE
:1007D400A80BA81AD82BA81FF42BA609A60A03193C
:1007E400A703A7092608A4002708A500281F00348A
:0C07F400A209A20A0319A303A309003400
:00000001FF
